:020000020000FC
:0200000038C006
:10000E004DC00D0A56657273696F6E2053414131B2
:10001E003035372D312E345043200D0A4269756C20
:10002E00642032302E30312E323030380D0A417588
:10003E00746F723A20416E6B7564696E6F762041F3
:10004E002E4E2E200D0A75613376766D406D6169E8
:10005E006C2E7275204B687A4552524F522048458D
:10006E004C4C4F571FED1DBF7894F0D2EFD210E2DB
:10007E0015BF5ED26ED294D2D3D26AE777E310E187
:10008E0085ED93E81AD210E1862F972F16D2ADD2B6
:10009E00CCD272D2C5D233278895FECF0FB61AB105
:1000AE001F771AB95F9BFECF4CB1493609F007C0D6
:1000BE0059D2B6D21AB110681AB90FBE1895463673
:1000CE0009F00BC092D2B1D257D274D2A9D2332733
:1000DE001AB110681AB90FBE1895413709F013C03E
:1000EE0011E020E0611B720B10E1862F972FE5D1F6
:1000FE007CD29BD241D25ED293D233271AB11068F2
:10010E001AB90FBE1895473709F013C011E020E059
:10011E00610F721F10E1862F972FCFD166D285D235
:10012E002BD248D27DD233271AB110681AB90FBE1E
:10013E001895413609F013C015E020E0611B720BD3
:10014E0010E1862F972FB9D150D26FD215D232D25D
:10015E0067D233271AB110681AB90FBE18954337F4
:10016E0009F013C015E020E0610F721F10E1862F19
:10017E00972FA3D13AD259D2FFD11CD251D23327C5
:10018E001AB110681AB90FBE18954A3709F013C084
:10019E001AE020E0611B720B10E1862F972F8DD194
:1001AE0024D243D2E9D106D23BD233271AB11068FA
:1001BE001AB90FBE1895483709F013C01AE020E09F
:1001CE00610F721F10E1862F972F77D10ED22DD28D
:1001DE00D3D1F0D125D233271AB110681AB90FBE78
:1001EE0018953395313041F0323061F0333081F073
:1001FE003430A1F03530C1F031D01AB110681AB9CF
:10020E000FBE189546D01AB110681AB90FBE1895C0
:10021E0085D01AB110681AB90FBE1895C4D01AB18C
:10022E0010681AB90FBE189503D133278EEC99E2D8
:10023E00680F791FA1D1BED1F3D110E185ED93E8FE
:10024E003CD110E1862F972F38D133271AB1106881
:10025E001AB90FBE1895680F791F0895142F7ED105
:10026E00403371F0413379F0423381F010E276D1B0
:10027E008DD1D6D133271AB110681AB90FBE189581
:10028E0060E070E0089560E177E2089560E27EE458
:10029E000895142F63D14033E1F04133D9F0423346
:1002AE00E9F04333F9F0443309F1453319F146339C
:1002BE0029F1473339F1483349F1493359F110E205
:1002CE004DD164D1ADD133271AB110681AB90FBE12
:1002DE001895089588EE93E0BEDF089580ED97E0BF
:1002EE00BADF089588EB9BE0B6DF089580EA9FE0C1
:1002FE00B2DF089588E893E1AEDF089580E797E1D5
:10030E00AADF089588E59BE1A6DF089580E49FE1CA
:10031E00A2DF089588E293E29EDF0895142F1ED186
:10032E004033E1F04133D9F04233E9F04333F9F091
:10033E00443309F1453319F1463329F1473339F185
:10034E00483349F1493359F110E208D11FD168D130
:10035E0033271AB110681AB90FBE1895089584E69E
:10036E0090E079DF089588EC90E075DF08958CE2D7
:10037E0091E071DF089580E991E06DDF089584EFDB
:10038E0091E069DF089588E592E065DF08958CEBD2
:10039E0092E061DF089580E293E05DDF089584E8E6
:1003AE0093E059DF0895142FD9D04033E1F0413353
:1003BE00D9F04233E9F04333F9F0443309F14533D0
:1003CE0019F1463329F1473339F1483349F14933AD
:1003DE0059F110E2C3D0DAD023D133271AB1106805
:1003EE001AB90FBE189508958AE090E034DF08958B
:1003FE0084E190E030DF08958EE190E02CDF0895E7
:10040E0088E290E028DF089582E390E024DF0895EB
:10041E008CE390E020DF089586E490E01CDF0895E1
:10042E0080E590E018DF08958AE590E014DF0895E6
:10043E00142F94D04033E1F04133D9F04233E9F038
:10044E004333F9F0443309F1453319F1463329F1B9
:10045E00473339F1483349F1493359F110E27ED02F
:10046E0095D0DED033271AB110681AB90FBE189581
:10047E00089581E090E0EFDE089582E090E0EBDEFB
:10048E00089583E090E0E7DE089584E090E0E3DEF7
:10049E00089585E090E0DFDE089586E090E0DBDEF3
:1004AE00089587E090E0D7DE089588E090E0D3DEEF
:1004BE00089589E090E0CFDE0895C39822E02A9552
:1004CE00F1F7C498C39A27E02A95F1F7C29A27E06C
:1004DE002A95F1F7C2980000880F991F10F0C49862
:1004EE0007C022E02A95F1F7C49A23E02A95F1F786
:1004FE0022E02A95F1F7C29A27E02A95F1F7C298E1
:10050E001A9549F722E02A95F1F70000C49AC3988C
:10051E000000000000000000C29A00000000000071
:10052E000000C29827E02A95F1F7C29AC39A08955F
:10053E001FEF17BBC29AC39AC49A08952FEF239543
:10054E00611B700B18F4610F701F08953FEFF7CF0A
:10055E00089519E119B918E91AB908955D9BFECFEE
:10056E001CB9089522E5E0E1F0E0C895E395102D61
:10057E00F5DF2A95D1F7089524E0E2E6F0E0C8957C
:10058E00E395102DEBDF2A95D1F7089525E0E6E6E9
:10059E00F0E0C895E395102DE1DF2A95D1F7089587
:1005AE0026E0ECE6F0E0C895E395102DD7DF2A950E
:1005BE00D1F7089580E09AE2A62FB72FA81BB90BAA
:1005CE000AF005C0332710E2C9DFE0DF089586EA9E
:1005DE0091E5A62FB72F8A1B9B0B0AF005C0332778
:1005EE0010E2BCDFD3DF089508956F937F938EECF6
:1005FE0099E2681B790B552707E210E19FDF122E57
:10060E0003E018EE9BDF222E00E014E697DF322E79
:10061E0000E01AE093DF422E562E7F916F910895DF
:10062E001DE09CDF1AE09ADF089510E3110E210EF3
:10063E00310E410E510E112D91DF122D8FDF132D24
:10064E008DDF142D8BDF152D89DF08951F932F93CA
:10065E0010E020E02A95F1F71A95D9F72F911F9106
:0A066E0008955F9BFECF1CB10895B4
:00000001FF
